:1000000080314F28080008007E1480314E01961E72
:100010000A280B2813288C1E0E280F281328A73116
:100020001A2780314D28161C162817281F280C1C4B
:100030001A281B281F28A631732680314D28161E2A
:10004000222823282B280C1E262827282B288031FD
:10005000022080314D280B1F2E282F284D28191ED5
:10006000322833283E280F1E362837283E284301E1
:100070006F088A006E080A0080314D28991E4128B9
:1000800042284D288F1E452846284D2844016C08DB
:100090008A006B080A0080314D287E1009008031EB
:1000A00051280D308400A7308500DA3086000030FA
:1000B00087000D30A631AF268031AA308400A730EA
:1000C000850054308600013087001A30A631AF26F3
:1000D0008031C4308400A7308500CE3086000130E6
:1000E00087001C30A631AF268031B83084009A30AA
:1000F000850020308600023087004530A631AF26CB
:100100008031EE30840098308500A03086000230C7
:1001100087002F30A631AF26803104308400903024
:10012000850020308600033087001430A631AF26CA
:100130008031FC01EF01A0308400003085002930BF
:10014000A631A9268031203084000130850034306A
:10015000A631A9268031A0308400013085002E30E0
:10016000A631A9268031CF308400023085001630B8
:10017000A631A92680317E1040018031BF28A731E9
:10018000382780314830F1001B30F200A631A32619
:100190008031E630F1002630F200A6319D26803114
:1001A0005C304101CC005130CB006030890BD62847
:1001B000CB0BD628CC0BD62800008B170B17400191
:1001C00014149414141594151416941614179417E3
:1001D0007E016410400115101A107E01E4104001E8
:1001E00095109A107E01641140011515A7317827EA
:1001F00080310030A731292780314501ED000D30D5
:100200004101CB00FB30890B0329CB0B03290032C2
:1002100045016D0803190D290E296E296D0A031970
:10022000122913296E290030A73129278031410175
:10023000C3000D304101CB00FB30890B1D29CB0BD6
:100240001D2900320130A731292780314101C20028
:100250000D304101CB00FB30890B2C29CB0B2C2915
:1002600000320230A731292780314101C1000D3011
:100270004101CB00FB30890B3B29CB0B3B290032E2
:100280000330A731292780314101C0000D304101E1
:10029000CB00FB30890B4A29CB0B4A2900320430B2
:1002A000A731292780314101BF000D304101CB002A
:1002B000FB30890B5929CB0B592900320530A73166
:1002C000292780314101BE000D304101CB00FB30B8
:1002D000890B6829CB0B682900327B29D130410179
:1002E000C3000630C200C101C10A8230C0006F30B5
:1002F000BF00BE01BE0A41014308A8002808CB0088
:10030000CC014B08F3004C08F4006430F1000030DD
:10031000F2009C314724803171084001B20072081C
:10032000B300890D893B8909B400B50001309D31C6
:10033000A2258031400135084301BB00400134084B
:100340004301BA00400133084301B90040013208BB
:100350004301B80041014208CB00CC014B084201E7
:10036000A50041014C084201A6004101410842019B
:10037000C300A301A4014301C401C5014201C2019C
:1003800025084001AA00420126084001AB00AC014B
:10039000AD010030F8000230F7007430F600A630EE
:1003A000F50041012808CB00CC01CD01CE014E085B
:1003B000F4004D08F3004C08F2004B08F1009031B6
:1003C0001820803174084001A9007308A800720841
:1003D000A7007108A60099314E21803140012908FB
:1003E000B5002808B4002708B3002608B200013081
:1003F0009D31A2258031400135084301BF004001F5
:1004000034084301BE00400133084301BD004001F0
:1004100032084301BC0000304101A3000030A200BB
:100420000030A1000030A000FF30A7312927803123
:100430004101C400FE30A731292780314101C500A8
:10044000FD30A731292780314101C6004608CB0085
:10045000CC01CD01CE014508CF00D0014F08D0001E
:10046000CF014F08D2005008D300D401D501440871
:10047000D600D701D801D9011030D635D70DD80D07
:10048000D90D890B3D2A5608D2075708D33D580885
:10049000D43D5908D53D5208CB075308CC3D5408EC
:1004A000CD3D5508CE3D4E08A3004D08A2004C0896
:1004B000A1004B08A0002308031D682A4030200239
:1004C0004230213B0F30223B031C672A682A712AE5
:1004D00000304101A3000030A2000030A100003034
:1004E000A0004101A601A701FC30A73129278031D6
:1004F0004101CB00CC014B08CC00CB0126084B04BA
:10050000A60027084C04A700FB30A731292780311B
:100510004101CB0026084B04A6002708A7002708A6
:10052000803ACB0083304B02031D982AE830260224
:10053000031C9B2A9C2A9F2A4101A601A701410175
:10054000AB01AA01A9014201C10140011714971092
:1005500004309E314D2680316A30F2000130F300C4
:100560000230F4000030F500A731E02780316F3011
:10057000F2000030F3000130F4000030F500A73144
:10058000E027803100304001A8000030A700003093
:10059000A6000A30A5000030F4000130F3008630D8
:1005A000F200A030F10041012308F8002208F70012
:1005B0002108F6002008F5009B31EC2380317408F7
:1005C0004001AC007308AB007208AA007108A900D2
:1005D0009A31FD22803140012508303E4301DE0082
:1005E00000304001A8000030A7000030A6000A300B
:1005F000A5000030F4000030F3002730F200103086
:10060000F10041012308F8002208F7002108F60054
:100610002008F5009B31EC23803174084001AC00C8
:100620007308AB007208AA007108A9009A31FD2274
:10063000803140012508303E4301DF000030400199
:10064000A8000030A7000030A6000A30A500003046
:10065000F4000030F3000330F200E830F100410113
:100660002308F8002208F7002108F6002008F5000A
:100670009B31EC23803174084001AC007308AB005F
:100680007208AA007108A9009A31FD228031400148
:100690002508303E4301E00000304001A800003052
:1006A000A7000030A6000A30A5000030F40000309A
:1006B000F3000030F2006430F10041012308F8003B
:1006C0002208F7002108F6002008F5009B31EC23F2
:1006D000803174084001AC007308AB007208AA00B6
:1006E0007108A9009A31FD22803140012508303E71
:1006F0004301E10000304001A8000030A7000030B5
:10070000A6000A30A5000030F4000030F3000030ED
:10071000F2000A30F10041012308F8002208F70036
:100720002108F6002008F5009B31EC238031740885
:100730004001AC007308AB007208AA007108A90060
:100740009A31FD22803140012508303E4301E2000C
:1007500000304001A8000030A7000030A6000A3099
:10076000A500410123084001AC00410122084001DD
:10077000AB00410121084001AA00410120084001CD
:10078000A9009A31FD22803140012508303E430105
:10079000E30003309E314D268031A030F20002305C
:1007A000F3001430F4000030F500A731E027803169
:1007B000DE30F2000130F3000630F4000030F500C6
:1007C000A731E02780310A304001A0000030A100AD
:1007D0006430F1000030F20041012708F4002608DF
:1007E000F3009C314724803172084001A300710856
:1007F000A2009B319823803140012008303E430104
:10080000DB000A304001A0000030A1000A30F100F6
:100810000030F20041012708F4002608F3009C3163
:100820004724803172084001A3007108A2009B3167
:100830009823803140012008303E4301DC000A301B
:100840004001A0000030A100410127084001A300A1
:10085000410126084001A2009B31982380314001CC
:100860002008303E4301DD0003309E314D268031AB
:10087000B430F2000230F3001430F4000030F50020
:10088000A731E0278031D830F2000130F300063084
:10089000F4000030F500A731E02780314201410328
:1008A000031D532C542C4E2E00304001A800003064
:1008B000A7000030A6000A30A5000030F400013087
:1008C000F3008630F200A030F10041012308F80067
:1008D0002208F7002108F6002008F5009B31EC23E0
:1008E000803174084001AC007308AB007208AA00A4
:1008F0007108A9009A31FD22803140012508303E5F
:100900004301DE0000304001A8000030A7000030A5
:10091000A6000A30A5000030F4000030F3002730B4
:10092000F2001030F10041012308F8002208F7001E
:100930002108F6002008F5009B31EC238031740873
:100940004001AC007308AB007208AA007108A9004E
:100950009A31FD22803140012508303E4301DF00FD
:1009600000304001A8000030A7000030A6000A3087
:10097000A5000030F4000030F3000330F200E8304E
:10098000F10041012308F8002208F7002108F600D1
:100990002008F5009B31EC23803174084001AC0045
:1009A0007308AB007208AA007108A9009A31FD22F1
:1009B000803140012508303E4301E0000030400115
:1009C000A8000030A7000030A6000A30A5000030C3
:1009D000F4000030F3000030F2006430F100410117
:1009E0002308F8002208F7002108F6002008F50087
:1009F0009B31EC23803174084001AC007308AB00DC
:100A00007208AA007108A9009A31FD2280314001C4
:100A10002508303E4301E10000304001A8000030CD
:100A2000A7000030A6000A30A5000030F400003016
:100A3000F3000030F2000A30F10041012308F80011
:100A40002208F7002108F6002008F5009B31EC236E
:100A5000803174084001AC007308AB007208AA0032
:100A60007108A9009A31FD22803140012508303EED
:100A70004301E20000304001A8000030A700003030
:100A8000A6000A30A500410123084001AC00410145
:100A900022084001AB00410121084001AA004101A8
:100AA00020084001A9009A31FD228031400125082B
:100AB000303E4301E30003309E314D268031A030AB
:100AC000F2000230F3001430F4000030F500A731DA
:100AD000E0278031DE30F2000130F3000630F40010
:100AE0000030F500A731E0278031410120084201A4
:100AF000A00041012008CB002108CC002208CD0035
:100B00002308CE000830CE36CD0CCC0CCB0C890B94
:100B1000832D4B084201A10041012008CB00210890
:100B2000CC002208CD002308CE001030CE36CD0CEC
:100B3000CC0CCB0C890B962D4B084201A200450131
:100B4000EE01EE0103306E02031CA72DA82DA92D86
:100B5000BC2D6E08203E8600013087000108F100A0
:100B60006E08FD3E98317220803101304101CB008A
:100B70004B084501EE07A22D0A304001A0000030CD
:100B8000A1006430F1000030F20041012708F400B8
:100B90002608F3009C314724803172084001A300ED
:100BA0007108A2009B319823803140012008303E1B
:100BB0004301DB000A304001A0000030A1000A30F0
:100BC000F1000030F20041012708F4002608F3008C
:100BD0009C314724803172084001A3007108A200B3
:100BE0009B319823803140012008303E4301DC00D6
:100BF0000A304001A0000030A10041012708400157
:100C0000A300410126084001A2009B3198238031B6
:100C100040012008303E4301DD0003309E314D2667
:100C20008031B430F2000230F3001430F4000030B0
:100C3000F500A731E0278031D830F2000130F30011
:100C40000630F4000030F500A731E0278031410183
:100C500026084201BF00410127084201C0004501AA
:100C6000EF01EF0102306F02031C372E382E392EB0
:100C70004C2E6F083F3E8600013087000108F100CE
:100C80006F08FB3E98317220803101304101CB006A
:100C90004B084501EF07322E4201C10141012A03F1
:100CA000031D542E8B319F2B8C31372C400147086C
:100CB0008039D1004735D800C61F5F2E602E612EC7
:100CC000581458080319652E662E762E580A031DEF
:100CD0006A2E6B2E732E0030C7000030C600003025
:100CE000C5000030C400C617C7017E2E0030C70003
:100CF0000030C6000030C5000030C4004308803911
:100D0000C8004808D1064335D900C21F882E892E55
:100D10008A2E5914590803198E2E8F2E9F2E590A88
:100D2000031D932E942E9C2E0030C3000030C20071
:100D30000030C1000030C000C217C301A72E003030
:100D4000C3000030C2000030C1000030C0004308C2
:100D5000420441044004031DAE2EAF2EC82E0030C5
:100D6000C7000030C6000030C5000030C40080302D
:100D7000C6047F30C7045108C8004808C7044708A4
:100D8000C3004608C2004508C1004408C000FF2F48
:100D90005808031DCC2ECD2ED62E0030C3000030B7
:100DA000C2000030C1000030C000FF2F5808C8004A
:100DB000C9014908CB0059084802CA00031CCB03EB
:100DC0004A087F3ED20000304B3DD3004708D00098
:100DD0004608CF004508CE004408CD000030C700CB
:100DE0000030C6000030C5000030C4000030D7001D
:100DF0000030D6000030D5000030D400D9013E2F9D
:100E000059080319042F052F1F2F0130CD35CE0DA2
:100E1000CF0DD00D890B062F0130C435C50DC60D81
:100E2000C70D890B0D2FD71F162F172F182F4414FE
:100E30000130D435D50DD60DD70D890B192F4308A8
:100E40005002031D2D2F42084F02031D2D2F410874
:100E50004E02031D2D2F40084D02031C302F312F51
:100E60003A2F57174008CD024108CE3B4208CF3BEE
:100E70004308D03B0130C8004808D9071A3059024E
:100E8000031C432F442F002F50084F044E044D04E1
:100E900003194B2F4C2F652F5414652F0130C43587
:100EA000C50DC60DC70D890B4F2FD71F582F592FB2
:100EB0005A2F44140130D435D50DD60DD70D890BDA
:100EC0005B2FFF30D207FF30D33DC61F682F692F3D
:100ED0004E2FD901D71F6D2F6E2F8A2FFF3054054B
:100EE000C800FF305505C900FF305605CA007F30E5
:100EF0005705CB004B084A04490448040319812FC5
:100F0000822F852FD901D90A8A2F441C882F892F37
:100F10008A2F822F590803198E2F8F2FB72F013058
:100F2000C4070030C53D0030C63D0030C73D471CFA
:100F30009A2F9B2FB72F4408C8004508C9004608C0
:100F4000CA004708CB000130CC00CB37CA0CC90C13
:100F5000C80CCC0BA52F4B08C7004A08C60049088F
:100F6000C5004808C4000130D2070030D33D530803
:100F7000803AC80080304802031DC02FFF30520263
:100F8000031CC32FC42FD12FFF304001D2000030EB
:100F9000D3000030C7000030C6000030C50000306C
:100FA000C40040015308803AC80080304802031D45
:100FB000DB2F013052020318DE2FDF2FEB2F400111
:100FC000D201D3010030C7000030C6000030C50098
:100FD0000030C400D10140015208D800581CF12F44
:100FE000F22FF42FC617F82F7F30C8004808C60527
:100FF0005836C7005108C8004808C704BF2E08006B
:10100000080041012D08031906280728CD2898312A
:10101000C42088314201C400B6284101A601A701BD
:1010200026084201BF00410127084201C0004001DB
:10103000A20122083F3E8600013087000108F1002E
:101040002208FB3E98317220883101304001A00017
:101050002008A20702302202031C2F28302819285A
:101060004101AD01CD2804309E314D2688316A30D2
:10107000F2000130F3000230F4000030F500A73137
:10108000E02788316F30F2000030F3000130F400C7
:101090000030F500A731E027883140010E195128B2
:1010A0005228632818154101AD010B304001A10001
:1010B0002630A0005D30890B5B28A00B5B28A10BBC
:1010C0005B280032CD281811532804309E314D265C
:1010D00088316A30F2000130F3000230F400003051
:1010E000F500A731E02788316F30F2000030F300BF
:1010F0000130F4000030F500A731E02788314001CD
:1011000010188328842886281A1453281A10532864
:1011100004309E314D2688316A30F2000130F300F0
:101120000230F4000030F500A731E02788316F303D
:10113000F2000030F3000130F4000030F500A73178
:10114000E027883140019A144101AD010B30400184
:10115000A1002630A0005D30890BAC28A00BAC2884
:10116000A10BAC28003240019A10CD284408400160
:10117000A000A1012108003A0319BF28CD282008AA
:10118000F13A03193328023A03190D28043A0319D6
:1011900065280F3A03198828CD280800003040013F
:1011A0000F1801304101B800380842014D060319FB
:1011B000DA28DB282829410138084201CD00410105
:1011C0003803031DE428E528072901309E314D2608
:1011D00088316230F2000130F3000230F400003058
:1011E000F500A731E0278831DA30F2000030F30053
:1011F0000230F4000030F500A731E02788312530B7
:10120000F600A830F70099311D21883128290130D6
:101210009E314D2688316230F2000130F3000230F9
:10122000F4000030F500A731E0278831C730F20024
:101230000030F3000230F4000030F500A731E02761
:1012400088312530F600A830F70099311D2188310A
:10125000003040018F1801304101B70037084201CA
:101260004C060319342935298229410137084201E6
:10127000CC0041013703031D3E293F29612901307C
:101280009E314D2688316830F2000130F300023083
:10129000F4000030F500A731E0278831DA30F200A1
:1012A0000030F3000230F4000030F500A731E027F1
:1012B00088312530F600A830F70099311D2188319A
:1012C000822901309E314D2688316830F20001308C
:1012D000F3000230F4000030F500A731E027883138
:1012E000C730F2000030F3000230F4000030F500A7
:1012F000A731E02788312530F600A830F700993172
:101300001D218831003040010F1901304101B60024
:10131000360842014B0603198E298F29DC29410129
:1013200036084201CB0041013603031D9829992953
:10133000BB2901309E314D2688316430F2000130E6
:10134000F3000230F4000030F500A731E0278831C7
:10135000C730F2000030F3000230F4000030F50036
:10136000A731E02788312530F600A830F700993101
:101370001D218831DC2901309E314D2688316430B1
:10138000F2000130F3000230F4000030F500A73124
:10139000E0278831DA30F2000030F3000230F40048
:1013A0000030F500A731E02788312530F600A8305D
:1013B000F70099311D218831003040018F1901302B
:1013C0004101B500350842014A060319E829E92917
:1013D000362A410135084201CA0041013503031D87
:1013E000F229F329152A01309E314D2688315830D3
:1013F000F2000130F3000230F4000030F500A731B4
:10140000E0278831DA30F2000030F3000230F400D7
:101410000030F500A731E02788312530F600A830EC
:10142000F70099311D218831362A01309E314D2631
:1014300088315830F2000130F3000230F4000030FF
:10144000F500A731E0278831C730F2000030F30003
:101450000230F4000030F500A731E0278831253054
:10146000F600A830F70099311D2188310030400185
:101470000F1A01304101B400340842014906031932
:10148000422A432A902A410134084201C9004101FD
:101490003403031D4C2A4D2A6F2A01309E314D26FC
:1014A00088316630F2000130F3000230F400003081
:1014B000F500A731E0278831DA30F2000030F30080
:1014C0000230F4000030F500A731E02788312530E4
:1014D000F600A830F70099311D218831902A01309B
:1014E0009E314D2688316630F2000130F300023023
:1014F000F4000030F500A731E0278831C730F20052
:101500000030F3000230F4000030F500A731E0278E
:1015100088312530F600A830F70099311D21883137
:10152000003040018F1A01304101B30033084201FD
:10153000480603199C2A9D2AEA2A410133084201E0
:10154000C80041013303031DA62AA72AC92A013076
:101550009E314D2688316030F2000130F3000230B8
:10156000F4000030F500A731E0278831DA30F200CE
:101570000030F3000230F4000030F500A731E0271E
:1015800088312530F600A830F70099311D218831C7
:10159000EA2A01309E314D2688316030F200013058
:1015A000F3000230F4000030F500A731E027883165
:1015B000C730F2000030F3000230F4000030F500D4
:1015C000A731E02788312530F600A830F70099319F
:1015D0001D218831003040010F1B01304101B20054
:1015E0003208420147060319F62AF72A442B410123
:1015F00032084201C70041013203031D002B012BB9
:10160000232B01309E314D2688315A30F2000130B3
:10161000F3000230F4000030F500A731E0278831F4
:10162000DA30F2000030F3000230F4000030F50050
:10163000A731E02788312530F600A830F70099312E
:101640001D218831442B01309E314D2688315A307E
:10165000F2000130F3000230F4000030F500A73151
:10166000E0278831C730F2000030F3000230F40088
:101670000030F500A731E02788312530F600A8308A
:10168000F70099311D218831003040018F1B013056
:101690004101B1003108420146060319502B512B7C
:1016A0009E2B410131084201C60041013103031D57
:1016B0005A2B5B2B7D2B01309E314D2688315C30BF
:1016C000F2000130F3000230F4000030F500A731E1
:1016D000E0278831DA30F2000030F3000230F40005
:1016E0000030F500A731E02788312530F600A8301A
:1016F000F70099311D2188319E2B01309E314D26F6
:1017000088315C30F2000130F3000230F400003028
:10171000F500A731E0278831C730F2000030F30030
:101720000230F4000030F500A731E0278831253081
:10173000F600A830F70099311D2188310800AA0170
:1017400043013B08F4003A08F3003908F200380876
:10175000F1004308F8004208F7004108F60040088D
:10176000F5009331BD238B3174084301C300730826
:10177000C2007208C1007108C00042012708400180
:10178000B200420128084001B300B401B5010030A5
:101790009D31A2258B3140013508C3003408C200B9
:1017A0003308C1003208C00043013F084001C700B0
:1017B00043013E084001C60043013D084001C50009
:1017C00043013C084001C4009D3117258B31031CA7
:1017D000EA2BEB2B372C4201A701A8014101260877
:1017E000013EA6000030273DA7000130CB000030AD
:1017F000CC000030CD000030CE002008CB072108FF
:10180000CC3D2208CD3D2308CE3D4E08A3004D0817
:10181000A2004C08A1004B08A0002308031D1A2CAD
:10182000403020024230213B0F30223B031C192C58
:101830001A2C232C00304101A3000030A2000030FC
:10184000A1000030A00041012708803ACB0083307E
:101850004B02031D2D2CE8302602031C302C312CAA
:10186000342C4101A601A7014201C101C10A410175
:101870002B03031D3C2C3D2C802CAB014201530853
:101880004001E300420152084001E200A030E400C0
:101890000F30E5009931FA218B3140016308EB00EC
:1018A0006208EA003C30EC000030ED0098319B20EB
:1018B0008B3140016B084501E60040016A08450193
:1018C000E500420143084101CB00CC014B08400137
:1018D000E20041014C084001E30045016608400177
:1018E000E500450165084001E4009931FA218B319A
:1018F000400163084301C500400162084301C40080
:10190000033042012E02203003192D02031C892CC2
:101910008A2CD22CAD01AE01430144084001B20033
:10192000430145084001B300B401B50100309D31C9
:10193000A2258B3140013508C7003408C6003308A2
:10194000C5003208C4004230C3003C30C2003D3004
:10195000C1007130C000863156268B3140014308EA
:10196000DD004208DC004108DB004008DA009C3161
:10197000A6248B3140015A084201C20001309E3139
:101980004D268B31E730F2000130F3000330F400D4
:101990000030F500A731E0278B3142014208A63123
:1019A000D4268B310B3042012C02B83003192B02A4
:1019B000031CDB2CDC2CE12CAB01AC01A631DD26B9
:1019C0008B3141012C080319E62CE72CCD2DAC01FD
:1019D000420126084001E300420125084001E200DF
:1019E000430143084001A700430142084001A6000B
:1019F000430141084001A500430140084001A40003
:101A00004030A3000F30A2002B30A1000230A00014
:101A10009531C5258B3140012308DD002208DC000B
:101A20002108DB002008DA009C31A6248B3140011C
:101A30005B08E5005A08E4009931FA218B31400136
:101A400063084201A400400162084201A300003083
:101A50004301C3000030C2000030C1000030C000AC
:101A60000A304001EA000030EB006430E200003050
:101A7000E300420124084001E5004201230840013F
:101A8000E4009931FA218B3140016308ED006208CE
:101A9000EC00993182218B3140016A08303E4301CC
:101AA000C600003040016B3D4301C7000A304001D1
:101AB000EA000030EB000A30E2000030E3004201AF
:101AC00024084001E500420123084001E400993167
:101AD000FA218B3140016308ED006208EC00993176
:101AE00082218B3140016A08303E4301C80000303A
:101AF00040016B3D4301C9000A304001EA0000305B
:101B0000EB00420124084001ED004201230840019E
:101B1000EC00993182218B3140016A08303E43014B
:101B2000CA00003040016B3D4301CB00E730860026
:101B30000230870006304101CB0000301E00CB0B85
:101B40009E2D430146084501E70043014808450131
:101B5000E80043014A084501E9002030EA0020304E
:101B6000EB002030EC0003309E314D268B312030CD
:101B7000F2000330F3001430F4000030F500A73118
:101B8000E0278B31E730F2000230F3000630F4003A
:101B90000030F500A731E0278B318831CE208B3122
:101BA0009031A8208B319E31F9268B3112304201C1
:101BB0002A02C03003192902031CDF2DE02D982EC4
:101BC000A901AA010030A631BC268B31A631B52669
:101BD0008B31003A0319ED2DEE2DE62DA631792635
:101BE0008B3172084101A5007108A4005830F20041
:101BF0000230F3000730F4000030F500A731E02791
:101C00008B3100304101250276300319240203187C
:101C10000A2E0B2E102E0030A631D4268B31912E99
:101C200000302502763003192402031C182E192EC9
:101C3000272E003025027930031924020318212EA3
:101C4000222E272E2A30A631D4268B31912E003019
:101C50002502793003192402031C2F2E302E3E2E2C
:101C6000003025027C30031924020318382E392E47
:101C70003E2E5430A631D4268B31912E00302502D1
:101C80007C3003192402031C462E472E552E0030AB
:101C900025027F300319240203184F2E502E552E93
:101CA0007E30A631D4268B31912E003025027F3034
:101CB00003192402031C5D2E5E2E6C2E00302502BB
:101CC0008230031924020318662E672E6C2EA8306A
:101CD000A631D4268B31912E003025028130031994
:101CE0002402031C742E752E832E003025028430AE
:101CF0000319240203187D2E7E2E832ED230A631A6
:101D0000D4268B31912E0030250284300319240211
:101D1000031C8B2E8C2E912EFF30A631D4268B31B6
:101D2000912E2530F600A830F70099311D218B3116
:101D3000173042013002703003192F02031CA12E0C
:101D4000A22E5A2FAF01B0010130A631BC268B3133
:101D5000A631B5268B31003A0319AF2EB02EA82E2E
:101D6000A63179268B3172084101A5007108A400C3
:101D70005130F2000230F3000730F4000030F5007B
:101D8000A731E0278B31003041012502763003195D
:101D900024020318CC2ECD2ED22E0030A631D4260C
:101DA0008B31532F00302502763003192402031C97
:101DB000DA2EDB2EE92E00302502793003192402B9
:101DC0000318E32EE42EE92E2A30A631D4268B31D7
:101DD000532F00302502793003192402031CF12E01
:101DE000F22E002F003025027C3003192402031844
:101DF000FA2EFB2E002F5430A631D4268B31532FD0
:101E0000003025027C3003192402031C082F092FFF
:101E1000172F003025027F30031924020318112FD9
:101E2000122F172F7E30A631D4268B31532F00303E
:101E300025027F3003192402031C1F2F202F2E2F71
:101E4000003025028230031924020318282F292F7D
:101E50002E2FA830A631D4268B31532F00302502E7
:101E6000813003192402031C362F372F452F0030F1
:101E7000250284300319240203183F2F402F452FD9
:101E8000D230A631D4268B31532F00302502843036
:101E900003192402031C4D2F4E2F532FFF30A63160
:101EA000D4268B31532F2530F600A830F700993116
:101EB0001D218B31883101208B314001101D612F94
:101EC000632F84314E2C4330F2000230F300073090
:101ED000F4000030F500A731E0278B3141014308C1
:101EE000A631D4268B312530F600A830F700993181
:101EF0001D218B313C30F2000230F3000730F4003A
:101F00000030F500A731E0278B3141014208A631AE
:101F1000D4268B312530F600A830F70099311D21E9
:101F20008B313530F2000230F3000730F40000301E
:101F3000F500A731E0278B3141014108A631D426B5
:101F40008B312530F600A830F70099311D218B31F7
:101F50002E30F2000230F3000730F4000030F500BC
:101F6000A731E0278B3141014008A631D4268B31BF
:101F70002530F600A830F70099311D218B3127302C
:101F8000F2000230F3000730F4000030F500A73112
:101F9000E0278B3141013F08A631D4268B31253013
:101FA000F600A830F70099311D218B312030F20066
:101FB0000230F3000730F4000030F500A731E027CD
:101FC0008B3141013E08A631D4268B312530F600F5
:101FD000A830F70099311D218B31C830F200023052
:101FE000F3000730F4000030F500A731E0278B3113
:101FF0004101A9019131CB218B31612F80314F28D3
:1020000042011D121D160800003410340034D23471
:10201000003482340034003400340034FF34FF34A0
:10202000FF34FF34003450340034023400340134BF
:102030004001A101F41F1D281E282B28F109F209D7
:10204000F309F409F10A0319F20A0319F30A03194F
:10205000F40AA101A10AF81F2E282F283E28F5090D
:10206000F609F709F809F50A0319F60A0319F70A38
:102070000319F80A0130F9007908A1060030A5001B
:102080000030A4000030A3000030A20074087304E4
:102090007204710403194D284E288F28A001A00A4C
:1020A0005C280130F135F20DF30DF40D890B522847
:1020B0000130F9007908A007F41F5F286028512833
:1020C0000130A235A30DA40DA50D890B612874085C
:1020D0007802031D752873087702031D752872089E
:1020E0007602031D752871087502031C782879286B
:1020F00082287108F5027208F63B7308F73B7408F2
:10210000F83B22140130F436F30CF20CF10C890B7D
:1021100083280130A002031D8E288F286028210803
:102120000319932894289F28A209A309A409A509A3
:10213000A20A0319A30A0319A40A0319A50A250868
:10214000F4002408F3002308F2002208F10008003C
:1021500040010D19AC28AD28B32804304201BB0062
:102160000030BC00B6284201BB01BC0140018D1902
:10217000BA28BB28C12808304201B9000030BA0093
:10218000C4284201B901BA0140010D1AC828C92862
:10219000CF280A304201B7000030B800D2284201EF
:1021A000B701B80139083B074001A00042013A08D5
:1021B0003C3D4001A1004201370840012007420197
:1021C000BD0038084001213D4201BE0036083E06F0
:1021D000031DEC2835083D060319EF28F028C52912
:1021E000A92902309E314D269031DC30F2000030BA
:1021F000F3000130F4000030F500A731E027903102
:102200002530F600A830F70099311D219031C529FD
:1022100002309E314D269031DD30F2000030F30067
:102220000130F4000030F500A731E027903125306F
:10223000F600A830F70099311D219031C5290230F0
:102240009E314D269031DE30F2000030F300013037
:10225000F4000030F500A731E02790312530F6007A
:10226000A830F70099311D219031C52902309E31E7
:102270004D269031DF30F2000030F3000130F400E1
:102280000030F500A731E02790312530F600A83066
:10229000F70099311D219031C52902309E314D261C
:1022A0009031E030F2000030F3000130F4000030F3
:1022B000F500A731E02790312530F600A830F7006F
:1022C00099311D219031C52902309E314D26903122
:1022D000E130F2000030F3000130F4000030F5008E
:1022E000A731E02790312530F600A830F70099316A
:1022F0001D219031C52902309E314D2690316F301D
:10230000F2000030F3000130F4000030F500A73196
:10231000E02790312530F600A830F70099311D21D3
:102320009031C52902309E314D2690316F30F20038
:102330000030F3000130F4000030F500A731E02751
:1023400090312530F600A830F70099311D219031E9
:10235000C5293E08003A0319AE2992293D08043ADE
:102360000319F1280C3A03190829023A03193629EE
:10237000063A03191F29023A03194D291C3A031979
:102380006429043A03197B29922942013E08B600C8
:102390003D08B50008004001AF01AF0A4101430804
:1023A0004001BB00410142084001BC00410141081D
:1023B0004001BD00410140084001BE0041013F080D
:1023C0004001BF0041013E084001C000B62BB901E9
:1023D000BA0100308400A8308500013F8A00003F28
:1023E0000A0091314001A0003908303E8600870183
:1023F000200881000130B9070030BA3D3A08803A20
:10240000A00080302002031D072A08303902031C77
:102410000A2A0B2AE929033040013706031D112A35
:10242000122AD02A410120084201A00041012008BF
:102430004001A000410121084001A1004101220802
:102440004001A200410123084001A3000830A33647
:10245000A20CA10CA00C890B272A20084201A10084
:10246000410120084001A000410121084001A100D4
:10247000410122084001A200410123084001A300BC
:102480001030A336A20CA10CA00C890B412A200805
:102490004201A2004001C1014108203E86000130F6
:1024A00087000108F1004108FD3E9831722091310A
:1024B00001304001A0002008C10703304102031C85
:1024C000622A632A4C2A3B08F100003098317220BE
:1024D000913141304001A000EE30890B6D2AA00BF4
:1024E0006D2A000040013C08F10001309831722053
:1024F000913141304001A000EE30890B7D2AA00BC4
:102500007D2A000040013D08F10002309831722020
:10251000913141304001A000EE30890B8D2AA00B93
:102520008D2A000040013E08F100033098317220EE
:10253000913141304001A000EE30890B9D2AA00B63
:102540009D2A000040013F08F100043098317220BC
:10255000913141304001A000EE30890BAD2AA00B33
:10256000AD2A000040014008F1000530983172208A
:10257000913141304001A000EE30890BBD2AA00B03
:10258000BD2A00004001AF014A30F2000230F300E2
:102590000730F4000030F500A731E0279131B62B69
:1025A00083303306031DD52AD62AB62B003084008B
:1025B000A8308500013F8A00003F0A0092314001A7
:1025C000B800972B3808BB004330F2000230F3000C
:1025D0000730F4000030F500A731E02791314001C9
:1025E0003808A631D42691312530F600A830F700FE
:1025F00099311D219131B62B3808BC003C30F200D6
:102600000230F3000730F4000030F500A731E02776
:10261000913140013808A631D42691312530F60099
:10262000A830F70099311D219131B62B3808BD0033
:102630003530F2000230F3000730F4000030F500CE
:10264000A731E027913140013808A631D4269131D5
:102650002530F600A830F70099311D219131B62BB5
:102660003808BE00B62B3808BF00B62B3808C000AB
:10267000B62B3808A000A101A201A3013708A400CD
:10268000A5012408A500A4012408A7002508A80086
:10269000A901AA013608AB00AC01AD01AE011030B2
:1026A000AB35AC0DAD0DAE0D890B502B2B08A7072C
:1026B0002C08A83D2D08A93D2E08AA3D2708A007F3
:1026C0002808A13D2908A23D2A08A33D230841016D
:1026D000A300400122084101A2004001210841015C
:1026E000A100400120084101A0005F30F20002304B
:1026F000F3000630F4000030F500A731E0279131F7
:1027000040013608A631D426913140013708A63160
:10271000D426913140013808A631D4269131253094
:10272000F600A830F70099311D219131B62B3508FC
:10273000A000A1012108003A03199F2BB62B200805
:10274000903A0319E22A013A0319FC2A033A0319C1
:10275000162B013A0319302B073A0319332B013A90
:102760000319362B0C3A0319392BB62B40012F08CD
:10277000031DBB2BBC2BE7290800740880394001DE
:10278000A8007435AA00F31FC62BC72BC82B2A1428
:102790002A080319CC2BCD2BDD2B2A0A031DD12BA4
:1027A000D22BDA2B0030F4000030F3000030F200BE
:1027B0000030F100F317F401E52B0030F400003095
:1027C000F3000030F2000030F10078088039A900F1
:1027D000290828060319ED2BEE2BEF2B2817783547
:1027E000A900F71FF42BF52BF62B29142908031940
:1027F000FA2BFB2B0B2C290A031DFF2B002C082C7A
:102800000030F8000030F7000030F6000030F5002E
:10281000F717F801132C0030F8000030F7000030F3
:10282000F6000030F5002A0829020318182C192C8C
:102830003F2C281F1C2C1D2C212C8030A000200890
:10284000A8062A08AB002908AA002B08A9007108CD
:10285000AB007508F1002B08F5007208AB00760894
:10286000F2002B08F6007308AB007708F3002B0882
:10287000F7007408AB007808F4002B08F800AB01EF
:102880002908A000A1012108A3002A082002A20013
:10289000031CA3032308803AA40080302402031DF4
:1028A000532C1A302202031C562C572C892C7408E6
:1028B000730472047104031D5E2C602C0130612CC2
:1028C00000304001AB000030F4000030F300003075
:1028D000F2000030F1002908AA00902C2B1C712C6A
:1028E000722C762C2B360138AB00782C0310AB0CF5
:1028F000711C7B2C7C2C7D2CAB170130A000F43795
:10290000F30CF20CF10CA00B7F2C0130A00020087E
:10291000AA07400129082A02031C8F2C902C6E2C38
:10292000281B932C942CCA2C2A08031D982C992C14
:10293000A22C0030F4000030F3000030F200003030
:10294000F100C42D7508F1077608F23D7708F33DD4
:102950007808F43D741CAD2CAE2C562D2B1CB12CDC
:10296000B22CB62C2B360138AB00B82C0310AB0CB4
:10297000711CBB2CBC2CBD2CAB170130A000F43754
:10298000F30CF20CF10CA00BBF2C0130A0002008BE
:10299000AA07562D7408803AA0007808803A2002D1
:1029A000031DDC2C77087302031DDC2C76087202F1
:1029B000031DDC2C750871020318DF2CE02C182D88
:1029C000FF30A000FF30A100FF30A200FF30A300C5
:1029D00071087502A4007208763BA5007308773B66
:1029E000A6007408783BA7002408A0072508A13D8D
:1029F0002608A23D2708A33D2308F4002208F3007F
:102A00002108F2002008F1008030A0002008A8066C
:102A1000AB09AB0A2B08031D0E2D0F2D202D013005
:102A2000F1070030F23D0030F33D0030F43D202D41
:102A30007508F1027608F23B7708F33B7808F43B1F
:102A40007408730472047104031D272D282D522D60
:102A50002B08031D2C2D2D2D522D0030F40000309D
:102A6000F3000030F2000030F100C42D0130F135E8
:102A7000F20DF30DF40D890B372DAB1F402D412DB9
:102A8000422D71142B1C452D462D492D0314AB0DE1
:102A90004B2D0310AB0D2A0803194F2D502D522D2D
:102AA0000130AA02F31F552D562D362DA901AB1F5B
:102AB0005A2D5B2D692D2B087F390319602D612D4F
:102AC000642DA901A90A692D711C672D682D692D36
:102AD000612D290803196D2D6E2D9B2D0130F107F5
:102AE0000030F23D0030F33D0030F43D741C792D90
:102AF0007A2D9B2D7108A0007208A1007308A20016
:102B00007408A3000130A400A337A20CA10CA00CF0
:102B1000A40B842D2308F4002208F3002108F200FE
:102B20002008F1002A0A0319962D972D9B2D0130BC
:102B3000A0002008AA072A0A03199F2DA02DA52D61
:102B40002A08031DA42DA52DB32D0030F40000305C
:102B5000F3000030F2000030F1002A08031DB12D0F
:102B6000B22DB32DA8012A1CB62DB72DB92DF31700
:102B7000BD2D7F30A0002008F3052A36F400A81FE1
:102B8000C22DC32DC42DF41708004001230880393D
:102B9000AD002335B300A21FCE2DCF2DD02D331481
:102BA00033080319D42DD52DE42D330A031DD92D57
:102BB000DA2DE22D0030A3000030A2000030A10089
:102BC0000030A000A217EC2D0030A3000030A200BE
:102BD0000030A1000030A00027088039A800280894
:102BE000AD062735AE00A61FF62DF72DF82D2E14B5
:102BF0002E080319FC2DFD2D0C2E2E0A031D012E6F
:102C0000022E0A2E0030A7000030A6000030A500DA
:102C10000030A400A617142E0030A7000030A60034
:102C20000030A5000030A4002E080319182E192E1C
:102C30001E2E3308031D1D2E1E2E272E0030A3002E
:102C40000030A2000030A1000030A000FF2F2008BB
:102C5000F100260898310120953172084001B90031
:102C60007108B8003808A800A901AA01AB012B0817
:102C7000B2002A08B1002908B0002808AF003908BE
:102C8000A800A901AA01AB012B08B7002A08B600C9
:102C90002908B5002808B4002108F100250898315A
:102CA0000120953172084001B9007108B800380858
:102CB000A800A901AA01AB012808AF072908B03D67
:102CC0002A08B13D2B08B23D3908A800A901AA0184
:102CD000AB012808B4072908B53D2A08B63D2B08E2
:102CE000B73D2208F100240898310120953172087F
:102CF0004001B9007108B8003808A800A901AA016C
:102D0000AB012808AF072908B03D2A08B13D2B08C0
:102D1000B23D3908A800A901AA01AB012808B407EF
:102D20002908B53D2A08B63D2B08B73D0830AF3518
:102D3000B00DB10DB20D890B972E2108F1002408BA
:102D400098310120953172084001B9007108B8002E
:102D50003808AF073908B03D0030B13DB23D20081A
:102D6000F100250898310120953172084001B90021
:102D70007108B8003808AF073908B03D0030B13DE0
:102D8000B23D0830AF35B00DB10DB20D890BC22E7A
:102D90002008F10024089831012095317208400183
:102DA000B9007108B8003808AF073908B03D0030E5
:102DB000B13DB23D2108F10026089831012095313E
:102DC00072084001B9007108B8003808B407390822
:102DD000B53D0030B63DB73D2208F10025089831D9
:102DE0000120953172084001B9007108B800380817
:102DF000B4073908B53D0030B63DB73D2208F100B3
:102E0000260898310120953172084001B9007108F7
:102E1000B8003808A8003908A900AA01AB01083099
:102E2000A835A90DAA0DAB0D890B102F2808B407E2
:102E30002908B53D2A08B63D2B08B73D2F08A80044
:102E40003008A9003108AA003208AB001830AB36B0
:102E5000AA0CA90CA80C890B272F2808B40729084D
:102E6000B53D2A08B63D2B08B73D0830AF35B00D4B
:102E7000B10DB20D890B362F33082E07A800A9011A
:102E8000A90D2808823EB800FF30293DB9005F2F08
:102E90000130B435B50DB60DB70D890B492FB21FF2
:102EA000522F532F542F34140130AF35B00DB10DC4
:102EB000B20D890B552FFF30B807FF30B93DB61F53
:102EC000622F632F482FAE01B21F672F682F842F08
:102ED000FF302F05A800FF303005A900FF30310575
:102EE000AA007F303205AB002B082A0429042804ED
:102EF00003197B2F7C2F7F2FAE01AE0A842F341C49
:102F0000822F832F842F7C2F2E080319882F892F3F
:102F1000B12F0130B4070030B53D0030B63D003070
:102F2000B73D371C942F952FB12F3408A8003508D2
:102F3000A9003608AA003708AB000130AC00AB3757
:102F4000AA0CA90CA80CAC0B9F2F2B08B7002A08C1
:102F5000B6002908B5002808B4000130B8070030D1
:102F6000B93D3908803AA80080302802031DBA2FE5
:102F7000FF303802031CBD2FBE2FC82F7F30400109
:102F8000B7008030B6000030B5000030B400F32F39
:102F900040013908803AA80080302802031DD22F52
:102FA000013038020318D52FD62FE12F0030400111
:102FB000B7000030B6000030B5000030B400AD01FD
:102FC000F32F40013808B300FF30B405FF30B505DA
:102FD0007F30B6050030B705331CEF2FF02FF12FEF
:102FE000B6173336B7002D08A8002808B7043708ED
:102FF000A3003608A2003508A1003408A00008008C
:103000000800F900F501F6017108F300F4017308F6
:10301000F7007408F800791C0E280F281328770889
:10302000F5077808F63D0130F735F80D890B1428BF
:103030000310F90C7908031D1E281F280B28760899
:10304000F2007508F1000800083042016E02031812
:103050002A282B28462841012F08B03E860001303F
:103060008700010842019A000130F0007008410118
:10307000AF0708302F02031C3E283F284028AF012D
:103080000130F00070084201EE0748284E01191285
:10309000080042016E0803194E284F2849284E01A6
:1030A000191A532854285828710842019A006F2889
:1030B000191241013008B03E8600013087007108C6
:1030C00081000130F2007208B00708303002031CA2
:1030D0006A286B286C28B00101304201EE024E01D3
:1030E00019160800F20050019E18772878287328D6
:1030F0001E1772089A0070309B009D0171089C0099
:10310000400103108B1F85288628872803148B1302
:1031100050011E1555309F00AA309F009E149E1826
:10312000922893288F281E114001031C9828992863
:103130009A288B1708004101C901CA0140016A1C85
:10314000A228A328AA286C084101C90740016D08DC
:103150004101CA3D01304001EC35ED0D890BAC2831
:103160000130EB36EA0C890BB1286A086B04031DA9
:10317000BA28BB289E2841014A084001EB004101C2
:1031800049084001EA00080041012D080319C92837
:10319000CA28C4282E08A03E8600013087000108F6
:1031A0004201C50041012E08A83E8600013087007B
:1031B0000108F2000130F1007108AE0708302E025C
:1031C000031CE328E428E528AE014E0199120130E2
:1031D0004101AD024E0199167208080000343234E4
:1031E000013418340034E73400340034003400343F
:1031F000FF34FF34FF34FF34003410340034023421
:1032000000340134003421340134F4340034E73420
:103210000034003400340034FF34FF34FF34FF3412
:103220000034103400340234003401345A34A534EC
:1032300004348034033400340234FA013929770825
:10324000F9007608F8007A087807840079080318EE
:10325000790A85000008F10002308400A83085005A
:10326000013F8A00003F0A0099310130F8007808D8
:10327000FA077708F2007608F100A7319127993113
:103280007A08F800F90172087902031D49297108CA
:103290007802031C4C294D291F29080000304001E9
:1032A000B1000030B0000030AF000030AE00261C8E
:1032B0005A295B2963292A08AE072B08AF3D2C0841
:1032C000B03D2D08B13D0130AA35AB0DAC0DAD0DB3
:1032D000890B64290130A936A80CA70CA60C890B10
:1032E0006B292908280427042604031D7829792935
:1032F00057293108A9003008A8002F08A7002E0878
:10330000A600080040016A086B040319882989296E
:10331000B7294101C901C90A97290130EA35EB0DE6
:10332000890B8E290130EE006E084101C90740016A
:10333000EB1F9B299C298D2940016B086D02031D01
:10334000A3296A086C02031CA629A729AB296A08CD
:10335000EC026B08ED3B0130EB36EA0C890BAC2933
:1033600001304101C902031DB629B7299C2940013A
:103370006D08EB006C08EA0008007C08A03E86009F
:1033800001308700810142011D1DC729C829D429A8
:103390007C08A03E860001308700811444016A0841
:1033A0008A0069080A00993142019D1CD829D9294F
:1033B000E5297C08A03E8600013087000115440104
:1033C00068088A0067080A0099317C08A03E8600D8
:1033D0000130870001080319EE29EF29F62944017D
:1033E00066088A0065080A009931F929A7315F2724
:1033F000993108004001E801E901620863040319FA
:10340000022A032A322AE701E70A0F2A0130E235AD
:10341000E30D890B072A0130E6006608E707E31F82
:10342000122A132A062A0130E835E90D890B142ADD
:1034300063086502031D1E2A62086402031C212A18
:10344000222A272A6208E4026308E53B6814013057
:10345000E336E20C890B282A0130E702031D312AEA
:10346000322A132A6908E3006808E20008004E01C6
:103470009912BD30F1001930F200A63191269A312F
:103480004E0119122430F1001830F200A6319726AF
:103490009A31083042019F0090309D0024309E00F8
:1034A000CF309B009C010030F1001830F200A631B3
:1034B00085269A310030F1001030F200A6318B26BB
:1034C0009A316F30F1002630F200A6317F269A3112
:1034D0004201C5014101B001AF0108304201EE00D7
:1034E000FC014101AE01AD014E01991608004001F9
:1034F0009A01990196019701980104309500F730DF
:103500009100FF309200BB309300FF3094007E01A9
:10351000D9017F30CE00C301E401F430B800DA01F4
:10352000E501C401B901CF01E601BA01C501D0012D
:10353000DB01FF30BB00FF30C600FF30D100FF30A1
:10354000DC000730E700FF30BC00FF30C700FF3071
:10355000D200FF30DD000F30E8004E0116160830B3
:103560007D0190001730CB0010307E01A6000800CE
:103570005A34A534053482340034953400345A3436
:10358000A534053482340034943400345A34A534DC
:10359000053482340034933400345A34A53405346D
:1035A00082340034923400345A34A53405348234E1
:1035B0000034913400345A34A53405348234003454
:1035C000903400345A34A534043480340334003445
:1035D00000345A34A5340534823401344034003484
:1035E0005A34A534053482340134303400345A342A
:1035F000A534053482340034993440012808270466
:10360000260425040319052B062B3F2BFB01FB0A7F
:10361000142B0130A535A60DA70DA80D890B0A2B7B
:103620000130FA007A08FB07A81F172B182B092B6B
:1036300028082C02031D262B27082B02031D262BEE
:1036400026082A02031D262B25082902031C292BE4
:103650002A2B322B2508A9022608AA3B2708AB3BB8
:103660002808AC3B0130A836A70CA60CA50C890B8A
:10367000332B0130FB02031D3E2B3F2B182B2C0854
:10368000A8002B08A7002A08A6002908A500080002
:1036900003104001961D031403184F2B522B4001B9
:1036A0009615542B4001961101304201B3070030AA
:1036B000B43D0130B1070030B23D0130AF070030FA
:1036C000B03D0130AD070030AE3D0130AB070030FA
:1036D000AC3D0130A9070030AA3D40018D1C712B83
:1036E000722B752B01304101A90040018D18792BF7
:1036F0007A2B882B41012903031D7F2B802B882BDC
:103700000130AA00A90101304201A7070030A83DFD
:103710000F3042013402A03003193302031C912BF5
:10372000922B972BB301B40101304101AC0008008A
:103730004001A501A31F9D2B9E2BA52BA209A30928
:10374000A20A0319A30AA501A50AA11FA82BA92B48
:10375000AE2BA009A109A00A0319A10A200821047F
:103760000319B32BB42BDD2BA401A40AC02B013009
:10377000A035A10D890BB82B0130FA007A08A407F7
:10378000A11FC32BC42BB72B21082302031DCA2B57
:1037900020082202031CCD2BCE2BD22B2008A20204
:1037A0002108A33B0130A136A00C890BD32B01309B
:1037B000A402031DDC2BDD2BC42B25080319E12BF0
:1037C000E22BE72BA209A309A20A0319A30A2308E3
:1037D000A1002208A000080000304001A300003032
:1037E000A2000030A1000030A0007408730472042D
:1037F00071040319FC2BFD2B3E2CA401A40A0B2CF5
:103800000130F135F20DF30DF40D890B012C01306F
:10381000F9007908A407F41F0E2C0F2C002C01309E
:10382000A035A10DA20DA30D890B102C74087802F0
:10383000031D242C73087702031D242C72087602C2
:10384000031D242C71087502031C272C282C312CF5
:103850007108F5027208F63B7308F73B7408F83BF1
:1038600020140130F436F30CF20CF10C890B322CDD
:103870000130A402031D3D2C3E2C0F2C2308F40024
:103880002208F3002108F2002008F1000800F701E7
:10389000F21F4B2C4C2C532CF109F209F10A03199D
:1038A000F20AF701F70AF41F562C572C602CF30983
:1038B000F409F30A0319F40A0130F5007508F70654
:1038C000F801F901710872040319672C682C972C10
:1038D000F601F60A742C0130F135F20D890B6C2CCF
:1038E0000130F5007508F607F21F772C782C6B2C49
:1038F0000130F835F90D890B792C72087402031D1B
:10390000832C71087302031C862C872C8C2C710865
:10391000F3027208F43B78140130F236F10C890B93
:103920008D2C0130F602031D962C972C782C7708ED
:1039300003199B2C9C2CA12CF809F909F80A0319EE
:10394000F90A7908F2007808F10008000310400134
:103950005C0D5D0DFB007B08031DAF2CB02CB92C5A
:103960000030DD000030DC000030DB000030DA0029
:10397000162D5A08DE005B08DF005C08E0005D08D9
:10398000E1001F30E136E00CDF0CDE0C890BC22CAD
:103990005E08FA00DC17FF30DA05FF30DB05FF3088
:1039A000DC050030DD059630FB02FB1FD82CD92C3E
:1039B000F12C7B08803A973E0318DF2CE02CE12C99
:1039C000B02C0130DD36DC0CDB0CDA0C890BE22C80
:1039D0000130DE005E08FB07031DEF2CF02CE12C0C
:1039E000062D20307B02031CF62CF72C012DB02C69
:1039F0000130DA35DB0DDC0DDD0D890BF92C0130E2
:103A0000FB027B08031D052D062DF82C7A080319EF
:103A10000A2D0B2D162DDA09DB09DC09DD09DA0A7E
:103A20000319DB0A0319DC0A0319DD0A0800003058
:103A300040014005C80000304105C9008030420502
:103A4000CA007F304305CB004B084A0449044804B0
:103A5000031D2B2D2C2D342D0030C3000030C2004F
:103A60000030C1000030C00000304405C800003004
:103A70004505C90080304605CA007F304705CB00A8
:103A80004B084A0449044804031D472D482D502D76
:103A90000030C7000030C6000030C5000030C40050
:103AA000C31F532D542D6C2D0030C8000030C900A9
:103AB0000030CA008030CB004008C8024108C93B32
:103AC0004208CA3B4308CB3B4B08C3004A08C2002C
:103AD0004908C1004808C000C71F6F2D702D882DF0
:103AE0000030C8000030C9000030CA008030CB0070
:103AF0004408C8024508C93B4608CA3B4708CB3BB7
:103B00004B08C7004A08C6004908C5004808C40059
:103B10008030C3068030C70647084302031D9A2D34
:103B200046084202031D9A2D45084102031D9A2DA5
:103B30004408400203189D2D9E2DA02D0310A12D99
:103B4000031408004001BA003A080319A82DA92D52
:103B5000BD2DB51FAC2DAD2DBD2D3209BC003309D7
:103B6000BD003409BE003509BF00BC0A0319BD0AF7
:103B70000319BE0A0319BF0AC52D3508BF00340852
:103B8000BE003308BD003208BC00350834043304DD
:103B90003204031DCC2DCD2DD62D0030B5000030C4
:103BA000B4000030B3000030B2004C2E9630BB00A1
:103BB000E42D0130B6003608BB070130BF36BE0C1D
:103BC000BD0CBC0C890BDE2DFE303F05031DE92D1D
:103BD000EA2DD92DFE2D0130B6003608BB07013085
:103BE000BC070030BD3D0030BE3D0030BF3D013060
:103BF000BF36BE0CBD0CBC0C890BF82DFF303F0549
:103C0000031D032E042EEB2D0E2E0130BB020130BE
:103C1000BC35BD0DBE0DBF0D890B082EBE1B112E70
:103C2000122E182E02303B020318172E182E052EC6
:103C30003B181B2E1C2E242EFF30BC05FF30BD056B
:103C40007F30BE05FF30BF050310BB0C3B08B6003C
:103C5000B701B801B9011830B635B70DB80DB90DB7
:103C6000890B2C2E3608BC043708BD043808BE0466
:103C70003908BF043A0803193E2E3F2E442EB51FC3
:103C8000422E432E442EBF173F08B5003E08B40015
:103C90003D08B3003C08B2000800FB00E22E6C3087
:103CA000F2000130F3000230F4000030F500A731DB
:103CB000E0279E31E530F2000030F3000130F400DF
:103CC0000030F500A731E0279E31E330F2000030EC
:103CD000F3000130F4000030F500A731E0279E31F9
:103CE000F82E6C30F2000130F3000230F4000030A6
:103CF000F500A731E0279E31E530F2000030F300F7
:103D00000130F4000030F500A731E0279E31E330A8
:103D1000F2000030F3000130F4000030F500A7316C
:103D2000E0279E31E430F2000130F3000330F4006C
:103D30000030F500A731E0279E31F82E6C30F200FC
:103D40000130F3000230F4000030F500A731E02725
:103D50009E31E430F2000030F3000130F400003016
:103D6000F500A731E0279E31E330F2000030F30088
:103D70000130F4000030F500A731E0279E31F82E25
:103D80006C30F2000130F3000230F4000030F50036
:103D9000A731E0279E31E630F2000030F300013019
:103DA000F4000030F500A731E0279E31E230F20048
:103DB0000030F3000130F4000030F500A731E027B7
:103DC0009E31F82E7B08F900FA017A08003A0319AF
:103DD000EA2EF82E7908013A03194F2E033A0319F7
:103DE000712E013A03199E2E073A0319C02EF82EA0
:103DF0000800003040018D1A01304101BC003C0830
:103E00003D060319042F052F4F2F3C08BD003C0829
:103E1000031D0B2F0C2F2E2F01309E314D269E316E
:103E20005630F2000130F3000230F4000030F500AB
:103E3000A731E0279E31C730F2000030F300023096
:103E4000F4000030F500A731E0279E312530F60060
:103E5000A830F70099311D219E314F2F01309E313E
:103E60004D269E315630F2000130F3000230F4004E
:103E70000030F500A731E0279E31DA30F200003043
:103E8000F3000230F4000030F500A731E0279E3146
:103E90002530F600A830F70099311D219E31003001
:103EA00040010D1B01304101BA003A083B060319DD
:103EB0005A2F5B2FA52F3A08BB003A08031D612F2C
:103EC000622F842F01309E314D269E315430F200F6
:103ED0000130F3000230F4000030F500A731E02794
:103EE0009E31C730F2000030F3000230F4000030A1
:103EF000F500A731E0279E312530F600A830F70005
:103F000099311D219E31A52F01309E314D269E31C4
:103F10005430F2000130F3000230F4000030F500BC
:103F2000A731E0279E31DA30F2000030F300023092
:103F3000F4000030F500A731E0279E312530F6006F
:103F4000A830F70099311D219E31003040018D1BB2
:103F500001304101B900390842014E060319B12F61
:103F6000B22FFF2F410139084201CE00410139082B
:103F7000031DBB2FBC2FDE2F01309E314D269E31FD
:103F80005E30F2000130F3000230F4000030F50042
:103F9000A731E0279E31C730F2000030F300023035
:103FA000F4000030F500A731E0279E312530F600FF
:103FB000A830F70099311D219E31FF2F01309E312D
:103FC0004D269E315E30F2000130F3000230F400E5
:103FD0000030F500A731E0279E31DA30F2000030E2
:103FE000F3000230F4000030F500A731E0279E31E5
:103FF0002530F600A830F70099311D219E310800C8
:104CDE00A7315F27A63108004E010C10A631F3262E
:104CEE00A631080041010D08F2000C08F100080081
:104CFE0072084401E6007108E500080072084401DC
:104D0E00EA007108E900080072084401E800710821
:104D1E00E700080072084401EC007108EB0008007F
:104D2E0072084301EF007108EE000800720843019B
:104D3E00EB007108EA00080072084301ED007108EB
:104D4E00EC000800640080010131890BAA2E0034AA
:104D5E00FE0012001E00FE0BB02E003403104101A7
:104D6E00131C03140030093D0800F10071084101C5
:104D7E009E009317131408004F0196019701980196
:104D8E0099019A019B010800623051018D008F013B
:104D9E0091010630930092010800F10042019E1C21
:104DAE00D92EDA2ED52E71089A0008001430F6008E
:104DBE00A830F70099311D21A631000008000130FE
:104DCE004101AB0042013208D3003108D200B101DB
:104DDE00B2014E010C10080043016A086B0403195E
:104DEE00F92EFA2EFF2E6B088A006A080A00A631E9
:104DFE0008004E010C100B140030F1000830F200C8
:104E0E00A6319D26A7314E01161408000034013438
:104E1E0006340534043403340234013480348234CD
:104E2E001B34053404344E018C1243016C086D049E
:104E3E000319222F232F282F6D088A006C080A00D1
:104E4E00A7310800F100640050019E182F2F302F5B
:104E5E002A2F1E1771089A0070309B001E141C0812
:104E6E000800A631C326A7319A317722A731A63181
:104E7E00CB26A731A7310027A731A7314B27A73162
:104E8E009A313722A7310800773040019F003D301C
:104E9E009D009C014E018C1296160330F1000030DD
:104EAE00F200A631A326A731803040019E000800F3
:104EBE007C08A83E86000130870042011908810057
:104ECE000130F0007008FC0708307C02031C702FC4
:104EDE00712F722FFC010130F00070084101AD07F7
:104EEE00080042018E018F01900191019201930100
:104EFE008D0141019E019B019C019401950196013A
:104F0E0097019A019901073098008430930002307E
:104F1E009D0008007208F5007108F4009A2F013008
:104F2E00F1070030F23D710884007208850012000E
:104F3E00031DA22FA32F962F74087102F10075087E
:104F4E00723BF20008000134133401341234013480
:104F5E002134013411340134143401341534013444
:104F6E001634013417340134183401341934013431
:104F7E002034033400345A34A53402342B340F3425
:104F8E004034A6347434023400343934A834203416
:104F9E002034203430343034303430343034303403
:104FAE003034303430340034503400340134003472
:104FBE000034F701F801F12F7708720786007808A0
:104FCE00733D87000108A631D426A7310130F707BB
:104FDE000030F83D7808803AF6007508803A76027F
:104FEE00031DFB2F74087702031CFE2FFF2FE32FE8
:104FFE000800C434183449341834003400340034F2
:10500E00003497342634BD341934913426340034A8
:10501E0000342434183437341A342D3420345334B5
:10502E0065346334753472346934743479342034AD
:10503E00543465347334743420342D340D340A34BE
:10504E000034483465346C346C346F342034573447
:10505E006F3472346C346434213420342534643427
:10506E000A3400345434723461346E3473346D3413
:10507E0069347434203474346534733474340A34BB
:0A508E0000340A346F346B34003430
:020000040001F9
:08000000FF3FFF3FFF3FFF3F00
:0A000E00EC3FFF3F9F3FFF3FFE3F26
:00000001FF
